:030000000219FDE5
:03000B000200AA46
:03002B000201626D
:03005B000202F8A6
:030073000202DEA8
:1000800002030406080C10182030406080040608A3
:100090000C10182030406080A0C000070F1F3F0DDB
:1000A0000D0403060D0502030202C2AFC0D0C0E07A
:1000B000206217E5256002E473E525F4F58A758B67
:1000C00000D262D0E0D0D0D2AF3285268AC262E5BB
:1000D00026F46030758B00D0E0D0D0C295C294C2B7
:1000E00093D2AF32C295C294C293206E0D20660A9D
:1000F0007405D5E0FDE57EF45290758B00D0E0D01C
:10010000D0D2AF32758A00C28DD26201FA01B93005
:100110006805206602D29501B9306805206602D2D2
:100120009401B9306805206602D29301B9D29230A9
:10013000680A2066077403D5E0FDD29501B9D29113
:1001400030680A2066077403D5E0FDD29401B9D265
:1001500090D29230680A2066077403D5E0FDD293EE
:1001600001B9C2AFC2AD53E6EFC0D0C0E0D2D3D226
:10017000AFC2CEE52A6007207449152A21C3780052
:10018000790020742EE580307E01F430E70278FF9C
:1001900053DACF207E0343DA20307E0343DA10C2E5
:1001A000D8C271E580307E01F430E70279FFC3E800
:1001B0009970CB306103752A40207403752A4088FA
:1001C0005FD27020740DE52B6004152B21D343DA28
:1001D00001C2D820700221E6A85F206102C270200F
:1001E000740221E488227882B60403852224C3E5C0
:1001F0002594404002D26420CF0AD0E0D0D043E61C
:1002000010D2AD32C2CF053A7802E52A60053074CB
:1002100002152AC3E55F94014005756200413075FF
:100220006300756C00E5622401F56250037562FF9E
:100230007982B7020D306D1DC3E5229432401685D8
:100240004D227982B7030E306D0BC3E52294324004
:1002500004798E8722C3E523952260084004152384
:1002600041640523D8CA056CE56C7002156CD56D28
:1002700063756D017805C3E56C956E4057C3E56CF9
:10028000956F50087801756D03020298C3E56C956F
:100290007050057801756D01C3E5659524401E79A0
:1002A00082B7040241C9206D14852465E56C0460A1
:1002B00003856E6C756D0175233C0202D4E56528DB
:1002C00050057565FF41C9F565E565047006756300
:1002D000FF756CFFD0E0D0D043E610D2AD32C2AF94
:1002E000C0D053E67FC260759100855694855795BE
:1002F000759104D0D0D2AF32C2AF53E6EFC2ADC0D9
:10030000D0C0E0C0F0D2D3D2AFA8FBA9FCC2D83095
:100310007102615F53DACF207E0343DA10307E032F
:1003200043DA20D271E580307E01F420E7026136A5
:1003300088278928A13E53DACF207E0343DA203074
:100340007E0343DA10C2D8C271307402A12A780049
:10035000E580307E01F430E702A12A885FA11253C4
:10036000DACF207E0343DA20307E0343DA10C271F5
:10037000206102813853DACF207E0343DA10307EC9
:100380000343DA20C2D8D271885A895BC3E89558F2
:10039000F8E99559F97B007E087A00C3E8948CE966
:1003A00094005005755E00812A882178A2E6A82174
:1003B0006055C3E894C8E994005008E4D2E4FB7A9D
:1003C0000A8105C3E89468E994015008E4D2E3FB8C
:1003D0007A0F8105C3E894D0E994025008E4D2E290
:1003E000FB7A1E8105C3E894A0E994055008E4D285
:1003F000E1FB7A3C8105C3E89498E994085008E44D
:10040000D2E0FB7A787E00C3E8955CFCE9955DFD5F
:1004100030E70AECF42401FCEDF43400FD755E00D5
:10042000C3EC9AED9E5003755E01885C895D855A28
:1004300058855B597802A112C3E89527F8E99528F9
:10044000F9307C0281F6307B0281F6307A0281EF4E
:10045000207502815BE9FDE8FC817AE9C313F9E8C4
:1004600013F830790281EFE9C313F9E813F8307813
:0F0470000281EFE9C313FDE813FC206126C3EC02
:10047F00941CED940240028191ED7018C3EC94C866
:10048F0050120529C3E529940A5002A12A755F006D
:10049F00D270A12AE529600215297400207F037804
:1004AF0096E624FAFEE43400FFC3EC9EFCED9FFDBC
:1004BF0050067800790081F6C3EC94FFED9400406C
:1004CF000678FF790081F6EC8575F0A4C5F0A2F7E8
:1004DF0033F87900400302051278FF790002051204
:1004EF00E9C313F9E813F8307C0EE9600278FFC313
:1004FF00E81338F8E43400F9C3E894FFE9940040B6
:10050F000278FF885FD270206102A12A741FF45510
:10051F002F4BF52FC274EB7002D274752A403074D2
:10052F0003752A0A306102A13E20740353DAFE20BC
:10053F007403752B20D0F0D0E0D0D0D2AD43E610AD
:10054F0032790102056E790302056E790A02056E92
:10055F00791E02056E796402056E79C802056E7800
:10056F0017E4D5E0FDD8FAD9F6227A147B78020584
:10057F00957A107B8C0205957A0D7BB40205957ADE
:10058F000B7BC80205957902B27DE4D291D5E0FDCF
:10059F00D294D5E0FDC294D5E0FDC291D5E0FDD255
:1005AF0095E576D5E0FDC2957496D5E0FDD9D9EAEB
:1005BF00F8D5E0FDD8FBDBCED29122C37C007D00C5
:1005CF0075F00005F0EA33FAEB33FB50F6EB13FB53
:1005DF00EA13FAC3E9FFE8FEE89AF8E99BF9500439
:1005EF00EFF9EEF8B3EC33FCED33FDD5F0DFEDF9B9
:1005FF00ECF822E889F08A20D2D4F8A9F07B0030F9
:10060F00F70B7BFFF42401F8E9F43400F9E88520B7
:10061F00F0A4ADF0F8E98520F0A4AFF0FEED2EF9CF
:10062F0074003FFA7C04C3EA13FAE913F9E813F8EC
:10063F00DCF48BF030F70AE8F42401F8E9F4340025
:10064F00F9E889F0C2D4F8A9F0227882B60403023F
:10065F0006F8C3E55F9419401EE52D540670182067
:10066F006D3678057994E7146007780A146002787C
:10067F0012C3E54198401F306D09856765756CFFA2
:10068F00756D01852224E4F545F546F547F548F5E6
:10069F0049C26D0206F8D26D7994E7147013E52301
:1006AF00F43333F913F8E9540104F9E854FE020660
:1006BF00ECE714147014E523F4333333F913F8E92A
:1006CF00540304F9E854FC0206F4E523F4333333FE
:1006DF0033F913F8E954070404F9E854F8C39440C4
:1006EF00F8E99400F98845894622C3E54113F9E5F5
:1006FF004013F8C3E54598F8E54699F9500CC3E85F
:10070F009480E994FF4016020730C3E8947FE99480
:10071F00005003020730787F790002073078807924
:10072F00FF884A894B22E54A2547F8E54B3548F9BA
:10073F00854B20E4300701F43549FA30E709C3EA65
:10074F0094F0401502076EC3EA940F500302076E30
:10075F0078FF79FF7A0F02076E780079007AF0C37D
:10076F00E5249564500AC374019524500B02078C3D
:10077F00E54B20E70E02078CE54B30E706884789EB
:10078F00488A492278A4E6FAC3E54A33F8E54B33A1
:10079F00F9D102E930E70BC3E89480E994FF4013E5
:1007AF00E1C6C3E8947FE994005002E1C6787F79EF
:1007BF0000E1C6788079FFE820E715C3E52398F8B4
:1007CF004009C3E8940140030207ED78010207EDE9
:1007DF00E8F424012523F840030207ED78FF884C45
:1007EF002278A5E6FAA848A949D102E930E70CC357
:1007FF00E89401E994FF4016020821C3E894FFE949
:10080F009400500302082178FF7900020821780133
:10081F0079FFE920E715C3E54C98F84009C3E89440
:10082F000140030208487801020848E8F424012532
:10083F004CF8400302084878FF88242278FFC264EE
:10084F0020693D206A12D264C3E541940A4009C36E
:10085F00E52594405002C26479A1E76023E5416029
:0D086F001F74FF8541F0848539F0306A0365
:10087C0075F005A4F8C5F0600278FFC3E8956750E1
:10088C0002A867886622C3E5409440E5419401E5DF
:10089C006650031401A3046002F566227883E6F522
:1008AC0020120F4575E89012055075E890E5E82088
:1008BC00ECFBA8BDA9BE120FE3757155757200C390
:1008CC00740013FD7455606613FC74552CFC740095
:1008DC003DFDECFAEDFBC3E89AE99B4014E571246D
:1008EC0055F571E5723400F572EA2CFAEB3DFB809C
:1008FC00E5AE71AF72C3E57213F9E57113F8C3E994
:10090C0013F9E813F87A03C3E913F9E813F8DAF7E3
:10091C00AA201A700975710075720002093A1AEA58
:10092C006008EE28FEEF39FFDAF88E718F722275AF
:10093C00E890227883E6FFE5E820ECF7A8BDA9BE95
:10094C000573C3E57394084052757300E9FA79A0F6
:10095C00E76044EA7007E574601B020975C3E8950B
:10096C00746010E5745006600C140209810460F97F
:10097C00020981E574F574C3946D401B7564C0C3A2
:10098C0094044013756480C39404400B756440C395
:10099C009404400375640075BB0622EFC394016098
:1009AC001F7455601BC3E894FFE994035012C3E80D
:1009BC009571E995725009E564600C15640209D3D0
:1009CC00E564F460020564A864C3E524985002A8A9
:1009DC0024C3E89565400AA865E565F46003856560
:1009EC006488258826E573B4070375BB102274321E
:1009FC0079A687F0A4C5F0A2F733F8C3E895644054
:100A0C0002A8648822882488258826886722754055
:100A1C00007541F022C2AF75C820A8CCA9CDAA3A66
:100A2C0030CF010A75C824D2AFAB3BAC3C883B89B4
:100A3C003CC3E89BF8E99C206908F93067026136F1
:100A4C004193AD3D8A3DF9EA9DFA600478FF79FF48
:100A5C00AE3EAF3F8B3E8C3FC3EC9FFCC3E99CF595
:100A6C0042A83BA93CC3E89EF8E99FF9C3E54113B2
:100A7C00FBE54013FAE82AF540E93BF541500675D1
:100A8C0040FF7541FF41DDAA40AB41AC40AD417E1A
:100A9C00047F02C3EB940440021E1FC3EB94084076
:100AAC00021E1FC3ED13FDEC13FCDEF7C3EA9CFA28
:100ABC00EB9DFBEF6009C3E913F9E813F8DFF7EAE4
:100ACC0028FAEB39FB8A408B4150067BFF8B408B1D
:100ADC0041C3EB94025002D2673069047F03610872
:100AEC007892E6FFC3E537948240110FC3E5379443
:100AFC00A040010FC3EF940640027F057E04E54140
:100B0C00C4540FF9E541C454F0F8E540C4540F281F
:100B1C00F8C3E89EFAE99400FB4009C3EA9402EB9F
:100B2C00940050047A02E4FB6182AA40AB41EBC40E
:100B3C00FEEAC4540F4EFCC3EA9CFAEB9400FBC3D0
:100B4C00E813C313F8EA28FAEB3400FB8A408B4114
:100B5C00C3EB94024002C2677804EBC4FE7B00EA4C
:100B6C00C4540F4EFAC3EA98FA4005C394025002DB
:100B7C007A027892E6FF3060026182855256855384
:100B8C0057D26043E680C3E49AF8E49BF9306702DD
:100B9C00811CE8FAE9FBD3E913FDE813FC885289C0
:100BAC0053C3EF94036038EF20E00DE82CF8E93DD7
:100BBC00F9ECFAEDFB020BD7E828F8E939F9C3E8B0
:100BCC002402F8E93400F97AFE7BFFC3EF9403406A
:100BDC000E8A548B55884E894F8C508D518150887C
:100BEC005489558A4E8B4F8C508D51306920C3E5FA
:100BFC003394034019E542A2E713F8E555F42401B8
:100C0C0038400B20E7087554FFF42401F55581504A
:100C1C00E8FAD3E813FC8852C3EF94036020EF206A
:100C2C00E007E82CF8ECFA813CE8282402F87AFE7C
:100C3C00C3EF940340088A54884E8C5081508854DA
:100C4C008A4E8C50E56BC3335002646BF56B30608D
:100C5C0002815A753402D26043E680E52D54066059
:0E0C6C0026A840A941C3E913F9E813F8C2AF66
:100C7A0053E67F759100C3E498F594E499F5957568
:100C8A009104D26043E680D2AF22D26575440075E2
:100C9A002000306B03752040020CB3D26575440006
:100CAA00752040306B03752000D2AF78012067228F
:100CBA00E52D54066002C265C3E5419405401378E8
:100CCA0002940540087803940540027806306902C8
:100CDA00780A206019E544601530690AC3E533943F
:100CEA00034003D53406D2AFD26CA1849162D2AF4D
:100CFA000000C2AF206726E541C3FB940F40027B88
:100D0A000FEB240530730123306A02742820620134
:100D1A0023F93069027982E58BC39940B50544E528
:100D2A009B5440B52002A16E30690A08C3E8940AB0
:100D3A0040010881DC20650281B3C26553E67F75F4
:100D4A0091003067107594007595FE759104D26014
:100D5A0043E68081B3AE40AF41C3E49EF594E49F7D
:100D6A00F595A155C3E5339402500281B33065026B
:100D7A0081B3D802A18281DCC26C53E67F759100EF
:100D8A00855494855595759104854E56854F57D24D
:100D9A006043E680D2AFE52D54066008206A02055A
:100DAA0033020DBE306C0D206B0A206507158115C4
:100DBA00810216162278003064053065027801E552
:100DCA003775F007A4F9E5F028F5F0E9A2F013A2C7
:100DDA00F113A2F213F537C394785003753778C329
:100DEA00E53795384008D266C295C294C2933060FE
:100DFA0002A1F8855056855157D26043E6802220D9
:100E0A007D11C2AF754302D291C292D2AF759F11C2
:100E1A00020FE0C2AF754302D291C290D2AF759F62
:100E2A0011020FE0307245207D22C2AF7543039054
:100E3A00013E757E02C293D290D292306204D2945D
:100E4A00C14EC291D2AF759F01020FE0C2AF754386
:100E5A000390013E757E02C295D292306204D2940A
:100E6A00C16EC291D2AF759F21020FE0207D17C2D9
:100E7A00AF754303900119C293306202D294D2AF84
:100E8A00759F01020FE0C2AF754303900119C29525
:100E9A00306202D294D2AF759F21020FE0207D11F9
:100EAA00C2AF754304D292C290D2AF759F21020F8E
:100EBA00E0C2AF754304D290D292C292D2AF759F6C
:100ECA0001020FE0307243207D20C2AF75430590C6
:100EDA00012D757E04C294D291306204D295C1EC80
:100EEA00C292D2AF759F11020FE0C2AF754305904F
:100EFA00014F757E01C294D291306204D293E10C03
:100F0A00C290D2AF759F11020FE0207D17C2AF7554
:100F1A00430590010FC294306202D295D2AF759FF9
:100F2A0011020FE0C2AF754305900123C2943062EB
:100F3A00EBD293D2AF759F11020FE0207D13C2AF9F
:100F4A00754306D290D292C291D2AF759F01020F19
:100F5A00E0C2AF754306D292C291D2AF759F210209
:100F6A000FE0307244207D20C2AF75430190014FDB
:100F7A00757E01C295D292306204D293E18AC29000
:100F8A00D2AF759F21020FE0C2AF75430190012DC8
:100F9A00757E04C293D290D292306204D295E1ACAB
:100FAA00C292D2AF759F01E1E0207D16C2AF7543B0
:100FBA0001900123C295306202D293D2AF759F216C
:100FCA00E1E0C2AF75430190010FC293306202D2D1
:100FDA0095D2AF759F01C2662290010D757E00C23F
:100FEA0095C294C293D292D291D290C26222788050
:100FFA0076070876070876010876040876FF0876E9
:10100A00FF08760A087602087601087601788C7657
:10101A00010876000876B40876FF0876FF0876FF9E
:10102A000876030876FF0876010876FF0876250811
:10103A0076D00876780876C80876040876FF0876A7
:10104A000108760008767A08760A08760108760199
:10105A000876000876FF227887E6FFC2727888C28F
:0F106A007DE630E102D27DC27E7889E630E10278
:10107900D27EC3EF94026008758E01D27302108E7E
:10108900758E00C273227880E6149000809378A44C
:10109900F67881E6149000809378A5F67886E614B0
:1010A90090008D9378A6F6789FE6F8700108C3E85A
:1010B900941140027811E82828F56E256E256E28CE
:1010C900F56F256E2828F570789CE67538FF753917
:1010D9000CB402067538A075390AB403067538824E
:1010E90075390578A3E61490009A93F569120FE310
:1010F90022227896E6FA7897E6FB7888E6B4030523
:10110900C3EB940EFB307F047A007BFFC3EB9AFCA0
:10111900C3948250027C827575000575EC8575F063
:10112900A4C3E5F0947D40F222D27F11FB12055F42
:101139007A007B007C10120555E55F2AFA74003BA2
:10114900FBDCF37C04C3EB13FBEA13FADCF7FEC206
:101159007F11FB22E5EF20E6037520000520903F73
:10116900FFE520146006901DFF14600093046003DE
:1011790075EF1253D9BF7581C043FF8012055075B1
:10118900EF0243B203E5B3240420E70DF521E5E3BB
:1011990020E0068521B343E301120FE37580FF7553
:1011A900A40075F19075D47F75908775A5BF75F208
:1011B900BF75D50075A60175E241E4F8F6D8FD754D
:1011C9006B01120FF812165E78988676753001C297
:1011D900AF12056912057912055F12058012055FC4
:1011E90012058712055F1217811205691205691226
:1011F9000564C2AF78FA79FA308707D9FBD8F702C4
:101209001C001161118F11FA11FB78988676120F63
:10121900E375885075891275C82475910475D8408D
:1012290075A82275B80275E690759B80759D007545
:10123900D10E75BC5875BB0675BA1175E8801205D3
:1012490050D2AF1208A853DACF207E0343DA2030F8
:101259007E0343DA1043DA01C2D8C271120569D29A
:10126900617B037A0CE55E70077A0CDB030211FBE4
:1012790012055F2070030211FBC270E55FC394027F
:1012890040E1E52F541F856160F561B560D5DAD578
:10129900C26153DACF207E0343DA20307E0343DA7A
:1012A90010C2D8C27178A2E67008D274E52F54E052
:1012B900F52FC275752900120564307409C3E52933
:1012C900940A4002D27512055578023074027800EA
:1012D900C3E55F9840F0C2AF12057912057912058E
:1012E90079D2AF120569754D00120555788CE6C3A0
:1012F900940150030213C8E530C39401500302134B
:10130900C8207435C3E55F94FF50030213C8C2AF08
:1013190012058ED2AF120564C3E55F940150EFC286
:10132900AF12057912055A120579D2AF120564C3B5
:10133900E55F94FF40E90218067F05D27F11FB1291
:101349000564C2AFC27F11FBAE5FC3E55F947FD274
:10135900AF4076120550C2AF12058ED2AFDFDC3135
:1013690032C3EE94057897F61205691216A0121782
:10137900897F0AD27F11FB120564C2AFC27F11FBBC
:10138900AE5FC3E55F947FD2AF50E6120550C2AF9E
:1013990012057912055A120579D2AFDFD63132EE2C
:1013A90024057896F61205691216A01217B81205C7
:1013B9006411FBC3E55F94FF5002610A021806C37A
:1013C900E55F954D4003855F4D1205647801798885
:1013D900E7B403027805C3E55F98400241F2C2AF62
:1013E90012058E12058E12058ED2AF12056975305F
:1013F90000E4F531F5320531E531F470390532781B
:101409009AE67819146012783214600D787D1460A8
:101419000878FA146003753200C3E532984017154D
:10142900327531B478998676C2AF12058ED2AF780B
:1014390098867612056412055AE52A7005307402F9
:1014490021FB78012074027806C3E55F9840A71252
:101459000564E52A70030211FBC2AF120FE3E4F53C
:0F14690022F523F524F525F526F56AD2AF78850F
:10147800E6C333F568E4F545F546F547F548F5491B
:10148800F573F52CF52DF53775730875BB10120536
:101498005012093BE5E820ECFBA8BDA9BEE97001A4
:1014A800F8887412093F75730875BB107887E6FED3
:1014B800760211617887EEF6C2AF7564FF1209FAF9
:1014C800852264852265852266D2AF75220175243E
:1014D8000175250175260185636C756D017888E6AF
:1014E800B40307C27D307602D27DD268D2697533E3
:1014F80000120F45120F6C120A1A120A21120A1A48
:10150800120A21120A1A02151DC2AF1161D2AF7553
:10151800730075BB06120CA5120659120DBF120EE8
:1015280009120A21120C94306D031206F920670380
:1015380012084B306703120892120DBF120E2E12BA
:101548000A21120CA5306D03120735120DBF120EB9
:10155800A7120A21120C94306D03120793120DBFC3
:10156800120ECE120A21120CA5306D031207F012CA
:101578000DBF120F45120A2112093B120C94120DCD
:10158800BF120F6C12093F120A2130692F206B2CF1
:1015980085676485676585636C756D0179187A0C54
:1015A800C3E533994009C269D26A8A350215C4C3B2
:1015B800E55F9401400302151D02161E306A1B20C8
:1015C8006B18E535147004C26AA111F535C3E55FDF
:1015D8009401400302151D02161E753600C3E5620C
:1015E8009401400985676585636C756D01C3E56283
:1015F80078FA985021307404E52A601A78F0306B34
:10160800058567647820C3E541985002A11D053619
:10161800E55F6002C121753600C2AF120FE378871B
:10162800E6FE760211617887EEF6E4F522F523F5F9
:1016380024F525F526F568C268D2AF120550120FB9
:10164800E3307406E52A700221FB788DE6C3940125
:10165800400241CF61FA901A0D78201216E2E52077
:10166800B4A50CA31216E2E520B45A0302168012A0
:101678000FF81216A002169F901A0378807B0A12A0
:1016880016E2A308DBF9901A0F788C7B181216E281
:10169800A308DBF9901A2722C2AF1217211216FBF2
:1016A800901A00740E1216E7A374041216E7A374B6
:1016B800141216E7901A0378807B0A1216E6A3081C
:1016C800DBF9901A0F788C7B181216E6A308DBF961
:1016D800121734121712901A2722E493F622E643BF
:1016E8008F01538FFD75EF0275B7A575B7F1F053EC
:1016F8008FFE22438F02438F0175EF0275B7A575E0
:10170800B7F1901A0DF0538FFC22901A0D74A5D1E1
:10171800E7901A0E745AD1E7227A3079D07820905F
:101728001A40D1E2E520F709A3DAF7227A3079D016
:10173800901A40E7D1E709A3DAF922AB77A878BB7A
:1017480001027980BB02027981BB03027982BB0462
:10175800027994BB05027983BB06027986BB07022E
:101768007992BB08027987BB0902799CBB0A027986
:1017780088BB0B027989E8F7227C05120569DCFB36
:1017880022C2AF12057912058012058712058E1242
:10179800055A12057912058012058712058E120561
:1017A8005A12057912058012058712058ED2AF22CA
:1017B800C2AF12058E12058712058012057912052F
:1017C8005A12058E12058712058012057912055ADC
:1017D80012058E120587120580120579D2AF22AE46
:1017E80077AF78C2AF12057912057912057912051B
:1017F8005ADEF212058E12055ADFF8D2AF221217FE
:10180800891217811217817577017578017579002A
:101818001217E77C05AD5F120569C3ED955F70F59A
:10182800C3E55F9401400AC3E55F94FF403702189F
:101838004A1217431216A0121789C2AF75EF121277
:101848001781DCD10579C3E5799403500280C11270
:1018580017810578E5771490009F93F808C3E57819
:0E18680098500280A81217811217810577C3CD
:10187600E577940C50028094120FF81216A0C2AFAE
:0618860075EF121217813C
:0319FD0002115D77
:101A00000E041407070104FFFF0A020101A55A0191
:101A100000B4FFFFFF03FF01FF25D078C804FF01DA
:081A200000FF0A010100FFFFB5
:101A400023585032354123202020202020202020E0
:101A500023424C48454C4923463333302320202031
:101A60002020202020202020202020202020202076
:101C0000C2AFC2D353D9BF7581C043B20343FF8073
:101C1000752438752503B1C975EF0275E24043F1AB
:101C20008053A47F75D400D2877DFA780379E67C4F
:101C300010752200752300901DD67B0675249875BB
:101C400025013087028142208708D8FBD9F9DCF7CB
:101C500081B4308708D8FBD9F9DCF781B4B189E4C5
:101C600093A3C39A6004DDC381B4DBDBB17B600264
:101C7000812B7B08E493FAA3B15CDBF87A30B15C8A
:101C8000752200752300B17BEAFCEBFDC3ED94FEE9
:101C9000400EB17B8A278B28ED30E0048A828B834B
:101CA000B17B7AC270D8C3ED94FE601350CEBD00F4
:101CB00025EC60097520007521FF0200008100A855
:101CC00027A9280809D804D90281D3B17FEA89AAB3
:101CD000F281C50D81A0C3ED94035049EDA2E092BD
:101CE000007AC5C3E5829400E583941C50902000DF
:101CF00010438F02438F0175B7A575B7F1F030001F
:101D00001FA827A9280809438F01538FFDD804D99C
:101D100002A12089AAE275B7A575B7F1F0A3A10DBC
:101D2000538FFC817C7AC1BD030CE493A3FAB140CC
:101D3000DCF8B138817C817EAA22AB23B15CEBFA5E
:101D4000EA6222752608C3E52313F523E52213F57D
:101D50002250066323A0632201D526EAB1C9B1C986
:101D600075260AEAF4200102D287300102C287B147
:101D7000C9C3134002C201D526EB22B17FEAFB2082
:101D80008702A17F308702A184752608AE24AF2583
:101D9000C3EF13FFEE13FEB1CDB1C9C3EA13308711
:101DA000024480FA30E703632201C3E52313F523DD
:101DB000E52213F52250066323A0632201D526D91C
:101DC000E52265236523F52222AE24AF250E0FDE22
:101DD000FEDFFCD20122424C48656C693437316326
:041DE000F3300601D5
:00000001FF
